:020000040000FA
:0A0000000000000093EF00F0A4D010
:08001800F7D09EA8FED7AD6EE3
:100020001200126E960E096E980E0A6E55D8D8B44C
:10003000CA90D8A4CA80FC0FD8A0CA92D8B0CA82ED
:10004000800E096E960E0A6E980E0D6E0E6ACAB07C
:1000500025D8CAB223D842D80904CB6E09C00BF008
:100060000AC00CF002500F6E106E023C106A4BD8A2
:100070000E50122E0AD0BE6E0C0EBD6E0DBEBD8A85
:100080000DBCBD889494CA841200BB6E0C0EBA6E6F
:100090000DBEBA8A0DBCBA889492F5D700D8D89014
:1000A0000D320A32093212000C6A0B6EFF0E0B265B
:1000B0000C2200D0D8A01200030E0A6EE60E02D861
:1000C000F5D70A6AFE0F096EE86A0A5AD8A012002C
:1000D0000000090600D0F8D70E6A0D6A100EF36E04
:1000E0000A340D360E360B500D5C0C500E5805E3DD
:1000F0000B500D5E0C500E5AD88009360A36F32E7E
:10010000EFD7095012000B500F02F3CF0DF0F4CFD0
:100110000EF00C500F02F3500E260B501002F3504D
:100120000E260D501200006AB8964F0EAF6EB06AE0
:10013000240EAC6E900EAB6E00010F0EC16E070E5A
:10014000B46EC69A470E926EE00E936EC00E946E19
:100150006ED0F2A409D0F294184A192AD6CF16F01C
:10016000D7CF17F0817A11009EAA19D0060EAB14D2
:1001700012E1E2CF30F0E1CF2FF0312A10EE42F061
:100180003150E126000EE222AECFE7FF30C0E2FFA1
:100190002FC0E1FF1100AE50AE50AB98AB881100FC
:1001A0003150325C14E0322AEACF0AF0E9CF09F08C
:1001B00000EE42F03250E926000EEA22EF502E6E99
:1001C0000AC0EAFF09C0E9FFD880120004D0E8683D
:1001D0002E6ED8A012001200316A326A9D8A9F8A60
:1001E000F28EF28C12009D9A00EE42F0010EF46E37
:1001F000F36AF306000EF45AEE6AF450F310F9E1D4
:10020000316A326A9D8A1200F29EE0CF42F2D8CF64
:1002100043F2E8CF44F2F28E0001A192F29E42C274
:10022000E0FF43C2D8FF44C2E8FFF28E1000949270
:100230008B9294948B94949A8B9A94988B98939A8B
:100240008A9A93928A9293968A96026A090E0C6E03
:100250008A0E0B6E020EE5DE026A090E0C6E8A0E25
:100260000B6E010EDEDE276A2790E2EC03F0939A14
:100270008A8A320E19DF939A8A9A00EE37F0080EB6
:10028000EE68E82EFDD72B6AA7DFADDFCD6AF294CA
:10029000F28A870ED56EB16AA192A082D08EA29208
:1002A000B00EB16EBD0EB9DE420EB7DE400EB5DE49
:1002B000D6CF16F0D7CF17F073DF2EC01AF0BE0ED0
:1002C0001A5C07E3FE0E1A5C02E344D102D01C6AFA
:1002D00041D11AAE21D01C6A8D0E1A5C05E11AC0FC
:1002E0001CF01D681E6817D09D0E1A5C05E11AC02F
:1002F0001CF01F6820680FD0AD0E1A5C05E11AC013
:100300001CF02168226807D0BD0E1A5C04E11AC0F7
:100310001CF0236824681CD11C5202E11BD118D1A7
:100320008D0E1C5CD8A441D01D2803E11AC01DF01D
:100330003AD01AC01EF0280E1D5C1FE1026A090E99
:100340000C6E8A0E0B6E020E6CDE1E520DE0D89003
:100350001E342D6E2DC002F0090E0C6E8A0E0B6E2F
:10036000010E5FDE8A8608D0026A090E0C6E8A0EC4
:100370000B6E010E56DE8A9615D0780E1D5C08E1D4
:100380002B908B9A3A683968386837683F800AD072
:10039000790E1D5C07E12B928B983E683D683C68A6
:1003A0003B683F801D68D6D0D3D09D0E1C5CD8A47E
:1003B000B6D01F2803E11AC01FF0AFD01AC020F03A
:1003C00020522AE1280E1F5C10E1026A090E0C6E11
:1003D0008A0E0B6E020E25DE026A090E0C6E8A0E64
:1003E0000B6E010E1EDE8A9615D0780E1F5C08E19A
:1003F0002B908B9A3A683968386837683F800AD002
:10040000790E1F5C07E12B928B983E683D683C6833
:100410003B683F801F689ED027A07ED0280E1F5CBF
:100420001CE1026A090E0C6E8A0E0B6E010E11ECB5
:1004300000F08A96D89020342C6E2C2A140E2C5C56
:1004400002E2140E2C6E2CC002F0090E0C6E8A0E05
:100450000B6E020E11EC00F05FD0780E1F5C2DE1E8
:100460008B8A2B807F0E205C22E220C040F001EEC0
:1004700042F0D8904034E926000EEA22EECF07F091
:10048000EFCF08F007501624036E08501720046EB3
:10049000000E1820056E000E1920066E03C037F0FE
:1004A00004C038F005C039F006C03AF004D03A680C
:1004B0003968386837683F802FD0790E1F5C2CE18F
:1004C0008B882B827F0E205C22E220C041F001EE5F
:1004D00042F0D8904134E926000EEA22EECF07F030
:1004E000EFCF08F007501624036E08501720046E53
:1004F000000E1820056E000E1920066E03C03BF09A
:1005000004C03CF005C03DF006C03EF004D03E689B
:100510003D683C683B683F801F681CD019D0AD0E19
:100520001C5C0AE1212803E11AC021F003D01AC0A3
:1005300022F0C1D80FD00CD0BD0E1C5C09E12328DD
:1005400003E11AC023F003D01AC024F0FBD802D074
:100550003FB076D8020E265CD8B065D03350165C1A
:10056000345017583550185836501958D8A05AD00A
:10057000368E26522AE12BB006D03A6839683868A0
:1005800037688B9A20D001EE42F0D8904034E926AB
:10059000000EEA22EECF07F0EFCF08F00750162446
:1005A000036E08501720046E000E1820056E000E12
:1005B0001920066E03C037F004C038F005C039F0CA
:1005C00006C03AF0827A2DD02CD0010E265C29E1AB
:1005D0002BB206D03E683D683C683B688B9820D0C3
:1005E00001EE42F0D8904134E926000EEA22EECF27
:1005F00007F0EFCF08F007501624036E08501720BD
:10060000046E000E1820056E000E1920066E03C041
:100610003BF004C03CF005C03DF006C03EF08278DF
:1006200000D00ED80CD019AC0AD0196A186A176A13
:10063000166A00EE37F0080EEE68E82EFDD738D6C1
:100640002668368E1B6A020E1B5C33E2D8901B3480
:10065000E96EEA6AEA36E936EA36370EE926000E2E
:10066000EA22EFCF03F0ECCF04F0ECCF05F0ECCFB3
:1006700006F03350035C345004583550055836505A
:10068000065815E2D8901B34E96EEA6AEA36E93674
:10069000EA36370EE926000EEA22EFCF33F0ECCF30
:1006A00034F0ECCF35F0ECCF36F01BC026F01B2A2F
:1006B000CAE33F901200780E215C20E12BA017D0F6
:1006C00022501624036E000E1720046E000E182010
:1006D000056E000E1920066E03C037F004C038F016
:1006E00005C039F006C03AF022C040F005D08B9A20
:1006F0003A683968386837683F8022D0790E215CC3
:100700001FE12BA217D022501624036E000E1720D3
:10071000046E000E1820056E000E1920066E03C030
:100720003BF004C03CF005C03DF006C03EF022C0E6
:1007300041F005D08B983E683D683C683B683F803F
:1007400021681200420E235C09E1245204E1279043
:100750008A9222D802D027808A8204D07B0E235C22
:1007600001E102D823681200949A8B9A94988B988E
:1007700093968A96026A090E0C6E8A0E0B6E010E13
:1007800011EC00F0026A090E0C6E8A0E0B6E020E5E
:1007900011EC00F02B6A12008B9A8B988A962B6AC8
:1007A0002C6A2D6A026A090E0C6E8A0E0B6E010EFF
:1007B00011EC00F0026A090E0C6E8A0E0B6E020E2E
:1007C00011EF00F00101E90E456FF80E446F740E51
:1007D000476FFC0E466F4D0E496FFD0E486F3A0E87
:1007E0004B6F7E0E4A6F2E0E4D6FCB0E4C6F260E4A
:1007F0004F6F4E69210E516F6D0E506F1D0E536F6E
:100800003F0E526F190E556F5469170E576F660ED3
:10081000566F150E596F450E586F130E5B6F7F0E96
:100820005A6F110E5D6F5C69100E5F6FB60E5E6FD2
:100830000F0E616F990E606F0E0E636F9F0E626FE9
:100840000D0E656FC30E646F0D0E676F666B0C0E39
:10085000696F500E686F0B0E6B6FB30E6A6F0B0EE5
:100860006D6F240E6C6F0A0E6F6FA30E6E6F0A0E03
:10087000716F2C0E706F090E736FC00E726F090EC0
:10088000756F5C0E746F090E776F766B080E796F5B
:10089000AA0E786F080E7B6F5B0E7A6F080E7D6F65
:1008A000110E7C6F070E7F6FCD0E7E6F070E816F6E
:1008B0008C0E806F070E836F500E826F070E856F50
:1008C000170E846F060E876FE20E866F060E896F15
:1008D000AF0E886F060E8B6F800E8A6F060E8D6FBF
:1008E000530E8C6F060E8F6F280E8E6F060E916F53
:1008F000906B050E936FD90E926F050E956FB50E26
:10090000946F050E976F920E966F050E996F710E8C
:10091000986F050E9B6F510E9A6F050E9D6F330EEB
:100920009C6F050E9F6F160E9E6F040EA16FFA0E40
:10093000A06F040EA36FE00EA26F040EA56FC60E8B
:10094000A46F040EA76FAE0EA66F040EA96F960ECD
:10095000A86F040EAB6F800EAA6F040EAD6F6A0E07
:10096000AC6F040EAF6F550EAE6F040EB16F410E3B
:10097000B06F040EB36F2E0EB26F040EB56F1B0E68
:10098000B46F040EB76F090EB66F030EB96FF70E92
:10099000B86F030EBB6FE60EBA6F030EBD6FD60EB7
:1009A000BC6F030EBF6FC60EBE6F030EC16FB70ED6
:1009B000C06F030EC36FA80EC26F030EC56F990EF2
:1009C000C46F030EC76F8C0EC66F030EC96F7E0E09
:1009D000C86F030ECB6F710ECA6F030ECD6F640E1E
:1009E000CC6F030ECF6F580ECE6F030ED16F4C0E2F
:1009F000D06F030ED36F400ED26F030ED56F340E3F
:100A0000D46F030ED76F290ED66F030ED96F1F0E4A
:100A1000D86F030EDB6F140EDA6F030EDD6F0A0E54
:100A2000DC6F030EDF6FDE6B020EE16FF60EE06F20
:100A3000020EE36FED0EE26F020EE56FE30EE46F60
:100A4000020EE76FDA0EE66F020EE96FD20EE86F64
:100A5000020EEB6FC90EEA6F020EED6FC10EEC6F66
:100A6000020EEF6FB80EEE6F020EF16FB00EF06F68
:100A7000020EF36FA90EF26F020EF56FA10EF46F66
:100A8000020EF76F9A0EF66F020EF96F920EF86F64
:100A9000020EFB6F8B0EFA6F020EFD6F840EFC6F61
:100AA000020EFF6F7D0EFE6F0201020E016F760EC9
:100AB000006F020E036F700E026F020E056F690E5B
:100AC000046F020E076F630E066F020E096F5D0E54
:100AD000086F020E0B6F570E0A6F020E0D6F510E4C
:100AE0000C6F020E0F6F4B0E0E6F020E116F460E43
:100AF000106F020E136F400E126F020E156F3A0E3A
:100B0000146F020E176F350E166F020E196F300E2E
:100B1000186F020E1B6F2B0E1A6F020E1D6F260E22
:100B20001C6F020E1F6F210E1E6F020E216F1C0E16
:100B3000206F020E236F170E226F020E256F120E0A
:100B4000246F020E276F0D0E266F020E296F090EFD
:100B5000286F020E2B6F040E2A6F020E2D6F2C6B66
:100B6000010E2F6FFC0E2E6F010E316FF70E306FDE
:100B7000010E336FF30E326F010E356FEF0E346FCF
:100B8000010E376FEB0E366F010E396FE70E386FBF
:100B9000010E3B6FE30E3A6F010E3D6FDF0E3C6FAF
:100BA000010E3F6FDB0E3E6F010E416FD80E406F9E
:060BB00000011200FFD756
:020000040030CA
:0300010006160ED2
:020005008580F4
:060008000FC00FE00F40E5
:00000001FF
